:020000020000FC
:100000004DCDA4C1000000001FC0000092C0000040
:1000100000009CC000000000000000000203040675
:10002000080C10182030406080000406080C1018DE
:100030002030406080A0C00000070F1F3F00050572
:100040000D050305030302004FB662FD0EC05520E7
:1000500009F00994C52DC095089483FDC795C4BDCA
:10006000C093A10064604FBE1895C09164000894CD
:1000700083FDC795C4BDC093A1006B7FC091640090
:10008000CF3F09F41FC070FF02C082FD05C04FBE04
:10009000C098AC9895981895C098AC98959875FDAF
:1000A0000DC065FD0BC0C9E0CA95F1F7C091B30062
:1000B000C0FDAB9AC1FDAD9AC2FD949A2092A100F9
:1000C0004FBE189524BCCC27C064C8BF6460F6CF6F
:1000D000C1CF70FFBFCF65FDBDCFC09ABBCF70FF52
:1000E000B9CF65FDB7CFAC9AB5CF70FFB3CF65FD83
:1000F000B1CF959AAFCFAB9870FFACCF65FDAACFCB
:10010000C7E0CA95F1F7C09AA5CFAD9870FFA2CF0E
:1001100065FDA0CFC7E0CA95F1F7AC9A9BCF949844
:1001200070FF98CF65FD96CFC7E0CA95F1F7959A15
:1001300091CF4FB6C9B7CF7EC9BF6E7FCCB5CE0DBC
:10014000DDB5DF1DDBBDCABD4FBE18953FB68F7E46
:10015000ABB7A074A2118061A0E0ABBFA9B7AE7F1E
:10016000A9BF7894A0916800AA2341F085FD2AC018
:10017000A0916800AA95A093680024C040E050E0D8
:1001800085FD14C0A0B396FDA095A2FD4FEFA3E09E
:1001900096FDA2E0A5BFAA27A064AABF8D7FA0B349
:1001A00096FDA095A2FD5FEF451741F7A8E161FD1F
:1001B000A093680085FD03C0A8E1A0936800409368
:1001C0009700816085FD0EC0A0916900AA2331F0DF
:1001D000A0916900AA95A093690004C08061AA2734
:1001E000A064AABF80FF38C0A09197004A2F61FF8A
:1001F0008E7F85FD18C0403F08F040EFA42FA295E8
:10020000AF704A0F5091B800533069F0A695A6958B
:1002100050FD01C0A69552FD03C0A41B4A2F03C088
:100220004A0F08F44FEFA091A0004A1708F44A2F94
:1002300040936100A72FA67079F0A0916D00A6955C
:10024000A69556E0A50F50916100A50FA0936100FF
:1002500018F4AFEFA0936100A0916100A093630038
:1002600040916300A0919C004A1708F04A2F542E39
:10027000A091A200AA2309F422C0542F5A1B10F403
:10028000A42F50E0BA2E8894AA1FAA2EA091A400F1
:10029000A095AA22A50E58F0A091A300A21509F0DE
:1002A000AA95AA0EA093A30048F04A2D08C0A091D9
:1002B000A300BA1608F0A395A093A3004FEF4093B4
:1002C00064007F7D485F08F07062A52DA03408F0BF
:1002D0006860A0916000A395A093600051F0F8942D
:1002E000A9B7A160A9BF84FF02C0A0E4ABBF3FBE15
:1002F0001895A0917400A395A093740041E05091CB
:100300006800552329F085FF03C05A955093680073
:10031000A0919700A13018F020929A000DC0209271
:100320009B002092A500A0919A00AF5FA0939A0035
:1003300018F0AFEFA0939A00F894A9B7A160A9BFF5
:1003400084FF02C0A0E4ABBF3FBE18953FB64CB5DA
:100350005DB58F7EABB7A074A2118061A0E0ABBF8A
:10036000A9B7AE7FA9BF789481FD23C0A2E096FD16
:10037000A3E0A5BF8260A0B396FDA095A2FF05C033
:1003800040936500509366003EC1A3E096FDA2E055
:10039000A5BFAA27A064AABF8D7F85FF01C026C183
:1003A00040E0A0B396FDA095A2FD20C14093970028
:1003B0000FC1A3E096FDA2E0A5BF8D7F61FF71C0D4
:1003C000A2E096FDA3E0A5BFAA27A064AABF826011
:1003D0004093920050939300A09090004A19B090DF
:1003E00091005B09BB24A22C4C38520518F42092D2
:1003F000960049C0A091D600AA2359F1483C520565
:1004000028F4A0E1BA2EAAE0AA2E23C04836A1E023
:100410005A0728F4A8E0BA2EAFE0AA2E1AC0403D31
:10042000A2E05A0728F4A4E0BA2EAEE1AA2E11C029
:10043000403AA5E05A0728F4A2E0BA2EACE3AA2E6F
:1004400008C04839A8E05A0720F4A1E0BA2EA8E76E
:10045000AA2EC42EA0919400CA1AD52EA091950060
:10046000DA0ADD202AF4AFEFC094D094CA1ADA0A6F
:1004700020929600A8E0A210A0E0CA14DA0618F4B0
:10048000A1E0A09396004093940050939500409172
:10049000920050919300409390005093910002E09D
:1004A00097C0A09165004A1BA09166005A0B94FD6D
:1004B00082C093FD80C092FD7CC086FF03C0D52E14
:1004C000C42E0CC05695479591FD73C0569547951F
:1004D00090FD6FC0D52EC42ED694C79461FD19C06F
:1004E000AC2DAC51AD2DA24008F005C0DD2089F443
:1004F000AC2DA85C70F4A0916700A395AA2311F01D
:10050000A0936700AA3008F471C020929700816020
:100510006DC0A0916700AA2319F0AA95A093670067
:10052000A22C5091BC0097FD06C0A090CA00533089
:1005300011F4A090D200AAEFAA0EA22DA21DCA18F3
:10054000DA0A4FB74170533049F4442321F087FD54
:1005500005C0806803C087FF01C08F77442359F02E
:10056000533031F4AFEFC094D094CA1ADA0A03C002
:1005700040E050E020C0533049F4CC0CDD1CAAE030
:10058000CA1AD20818F4A0E0CA2ED22CAFEFCA16AD
:10059000D20418F04FEF50E00EC0A091AE00CA9EFA
:1005A000412D000C441F50E008F012C04FEF50E006
:1005B0000FC05695479594FF07C0552309F04FEF9C
:1005C000A42FA6954A0F521D4F3F520508F04FEF3A
:1005D00040939700816061FF09C0AFE1A095A92316
:1005E000AB299A2F8F7DBB2009F48062A8E1A093EC
:1005F000680085FF03C0AAE0A093680061FD03C006
:1006000085FD01C08F7E85FD03C0A6E0A093690033
:10061000F894A9B7A160A9BF84FF02C0A0E4ABBF52
:100620003FBE189511E00AC013E008C01AE006C0EA
:100630001EE104C014E602C018EC00C005E1BB27AF
:10064000BA95F1F70A95D9F71A95C1F708952AE3F3
:1006500038E709C020E33CE806C02AE234EB03C0D7
:1006600025E238EC00C012E095FD9F7D95FF906279
:10067000BB27AD98BA95F1F7AC9ABA95F1F7AC985B
:10068000BA95F1F7AD9ABA95F1F7C09AB091AF006B
:10069000BA95F1F7C098B7E8BA95F1F71A9521F72E
:1006A000022FB22FBA95F1F70A95D9F73A95D9F6F4
:1006B000AD980895221B39E0001F3A9509F408957A
:1006C000221F211B18F4210F8894F6CF0894F4CF31
:1006D000622C722CB0E08894B395221F331FE0F790
:1006E000379527958894912E802E020B130B10F4CA
:1006F000192D082D10F4889401C00894661C771CED
:10070000BA9571F7172D062D0895322D11232AF46D
:100710003A9500951095031B130BF894029F712CCA
:10072000002D129F912C802C7894780C172D921C00
:10073000292DB4E06B2E2695179507956A94D9F765
:10074000332321F000951095031B130B0895089592
:1007500010917B00169500917A000795B0917F006B
:10076000B01B0B2FB0918000B10B1B2F28F4003869
:10077000BFEF1B0740F009C00F37120508F405C092
:100780000FE710E002C000E81FEF00938400109311
:100790008500089500918400B09181000B0F1091A5
:1007A0008500B09182001B1F20E03091850033232B
:1007B0000AF42A95B09183002B1F1AF4203F40F0D1
:1007C0000AC02F3008F407C00FEF1FEF2FE003C05F
:1007D00000E010E020EF30916300B0919C003B17E7
:1007E00018F4323030F009C0B0918500BB235AF0C4
:1007F00004C0B0918500BB2332F4009381001093B4
:1008000082002093830008952091D80000918400F5
:10081000000F10918500111F78DF11232AF4003892
:10082000BFEF1B0740F009C00F37120508F405C0E1
:100830000FE710E002C000E81FEF002352F0B09174
:100840006200B01B0B2F18F0013008F00AC001E065
:1008500008C000950F5FB09162000B0F08F001C057
:100860000FEF0093860008952091D9000091820037
:10087000109183004ADF11232AF40130BFEF1B07D8
:1008800040F009C00F3F120508F405C00FEF10E05B
:1008900002C001E01FEF112352F0B0918600B01B9F
:1008A0000B2F18F0013008F00AC001E008C00095D5
:1008B0000F5FB09186000B0F08F001C00FEF00939F
:1008C000630008950FEF677F71FD29C072FD09C0B5
:1008D0006860B0917B00BA3020F0B52DB03408F4D8
:1008E000677FB091D500BB23D1F0B0917B00BB23D3
:1008F000B1F00FEF10917B00DDDEF894B091730042
:1009000072FDB5E00B9F112D002D7894112309F095
:100910000FEFB0919F000B1710F400919F00009310
:100920009E00089500917A0010917B0000541140C0
:10093000B0919E0010F4BA9501C0B39511F0B09338
:100940009E00089500C008952091B700B6B1B6FD8D
:10095000FBCF04B115B1B6B1BF77B6B9B091AC0059
:10096000B395B093AC00B83060F12092AC00B09178
:10097000D400BB2321F1112329F0B091AD00BF3F7A
:1009800061F009C0B091AD000B1739F020F4BB2322
:1009900021F0BA9502C0B395E1F300919C00B093A9
:1009A000AD00B13A50F400ECB43938F400E8B7388F
:1009B00020F400E4BA3708F400E000939C00777F4D
:1009C0000895B0919C00B39511F0B0939C00B09144
:1009D000AC00B73009F47860089502E3F894B09160
:1009E000DA000B9F012D000C001F7894B0919C0041
:1009F0000B1710F000919C000093610000936300BE
:100A0000502E0093640000939F00089520927A0076
:100A1000B0EFB0937B000895F8940CB51DB520910C
:100A200074007894309175006090760000937500A2
:100A300010937600031B160971FD03C076FD81C07B
:100A40002BC070907700209377002709222311F0A4
:100A50000FEF1FEF8090780090907900309378002E
:100A6000609279006918161910937C000091750046
:100A7000109176000819190920917A0030917B00B5
:100A800036952795020F131F10F40FEF1FEF0093F9
:100A90007A0010937B0029C020917A0030917B006E
:100AA0003901B4E08B2EB2E09B2E343010F08A94E2
:100AB0009A94383010F08A949A94769467948A9431
:100AC000E1F726193709992021F0169507959A9490
:100AD000E1F7200F311F20937A0030937B0028F438
:100AE0003FEF30937A0030937B00323008F470642B
:100AF00071FF02C0B3E00DC0B091C600009171005B
:100B0000023838F0B395003A08F0B395B63008F0E3
:100B1000B5E09B2EB4E08B2E10917B0000917A0003
:100B200024E0169507952A95E1F70819120928F08F
:100B3000B02FB250B12FB20910F402E010E09801CA
:100B400026C020917A0030917B0039017694679419
:100B50006694669466942619320906950695200FC8
:100B6000321D20937A0030937B00323008F07F7B77
:100B700004E0369527953695279526952695201BD2
:100B800010F0223008F422E089019090C60060FD48
:100B9000FECFE0908C00F0908D006160B9B7B0613D
:100BA000B9BF380176FD44C07694679400938C00F9
:100BB00010938D00B92DB330E1F0B0FD04C0060DE7
:100BC000171D930106C0000F111F0250120922E0E9
:100BD00030E0B92DB33068F020938E0030938F0051
:100BE000009388001093890060928A0070928B00B5
:100BF0003DC000938E0010938F00209388003093A7
:100C0000890060928A0070928B0071FF10C0B091D1
:100C10006D00B33060F000918F0010917C0015954D
:100C2000010F28F022F020928E0000938F001EC04A
:100C3000669400938C00B92DB33091F0B0FD03C0E1
:100C4000060D262D03C0000F025022E0B92DB3304F
:100C500038F020938E000093880060928A0006C0CE
:100C600000938E002093880060928A0000917D009E
:100C700002FD0350013029F495FD0AC0B0E0B7B978
:100C800009C0023019F4B7E0B7B904C095FDF6CF3A
:100C9000B6E0B7B90091A400000F10F4BBE60B2733
:100CA0000093A40060FDFECFB2E0B0936E006160DF
:100CB000B9B7B061B9BFB72FB670A1F020917A0073
:100CC00030917B0036952795F8940CB51DB5020F31
:100CD000131F1BBD0ABD6160B0E1B8BFB9B7B061F9
:100CE000B9BF78940895606120927E0020E067FD8E
:100CF00020E206C0606120927E0020E267FD20E0D5
:100D0000789401E076FD11C0B72FB67009F06F7EC0
:100D1000B0917B00B55048F002E0B55020F003E000
:100D2000B55008F006E071FD0AE060FD12C0B09118
:100D30007E00BB2371F071FF08C0B0916D00B3302D
:100D400020F0B0916E00BA9519F4789470615CC08F
:100D5000AEDF789400000000F89476FD16C0109184
:100D60007B00173008F017E0B5E01B0F72FD10E1B3
:100D700083FF110F62FF110F71FD12E8B4B560908F
:100D8000A100B61990F2B10B80F2B0B7B77FB0BF37
:100D9000B8B1B0B7B860B0BFB0917E00B395B093B2
:100DA0007E00B8B176FD06C0B1E071FDB2E0BA9543
:100DB000F1F7B8B1B072B21709F01BC071FF05C0EE
:100DC00003950A3008F00395B0CF64FF99CF6F7E8A
:100DD0003CB56DB470907A0080907B00370D681C34
:100DE0006BBC3ABD6160B0E1B8BFB9B7B061B9BF23
:100DF00087CFB0916D00B23008F482CF64FD80CF10
:100E00000A9509F092CF7F7E20918E0030918F005D
:100E1000F894B0E1B8BF0CB51DB5020F131F1BBD90
:100E20000ABDE0908800F09089006160B9B7B061B8
:100E3000B9BF7894B72FB67039F0B0916D0072FFDA
:100E4000B395B0936D0009C074FF07C067FD05C07E
:100E500064FD03C0BF91BF91E1C4089500E063FF4A
:100E600003C064FF01C001E0F89410917100B7E085
:100E70001B9F212D102D7894200F269517952695D0
:100E800017952695179510937100183718F4B8E741
:100E9000B093710000917100B09172000B1720F0B7
:100EA0006062C098AC98959860FDFECFE0908A0093
:100EB000F0908B006160B9B7B061B9BF0895C49A72
:100EC000B2E095FD07C0F894B0937D00AD98AB9A61
:100ED0007894EAC0F894B0937D00AD98949A789491
:100EE000E3C0C498B3E082FF24C095FD11C002E0C6
:100EF000F894B0937D00E5E8F0E00093B300959896
:100F0000949862FF02C0AC9A01C0AD9A7894CCC0AC
:100F100002E0F894B0937D00E5E8F0E00093B300C0
:100F2000C098AB9862FF02C0AC9A01C0AD9A7894A9
:100F3000BBC095FD0BC0F894B0937D00EFE6F0E0E8
:100F4000959862FF01C0AC9A7894AEC0F894B093C3
:100F50007D00EFE6F0E0C09862FF01C0AC9A7894A3
:100F6000A3C0C49AB4E095FD07C0F894B0937D0087
:100F7000AB98949A789498C0F894B0937D00949824
:100F8000AB9A789491C0C498B5E082FF24C095FDD7
:100F900011C001E0F894B0937D00EBE7F0E000931E
:100FA000B300AC98AD9862FF02C0C09A01C0AB9A82
:100FB00078947AC004E0F894B0937D00EFE8F0E014
:100FC0000093B300AC98AD9862FF02C0959A01C03F
:100FD000949A789469C095FD0BC0F894B0937D0005
:100FE000E9E6F0E0AC9862FF01C0C09A78945CC07A
:100FF000F894B0937D00E5E7F0E0AC9862FF01C0A3
:10100000959A789451C0C49AB6E095FD07C0F894BB
:10101000B0937D009498AD9A789446C0F894B093BC
:101020007D00AB98AD9A78943FC0C498B1E082FF40
:1010300024C095FD11C004E0F894B0937D00EFE862
:10104000F0E00093B300C098AB9862FF02C0959A9D
:1010500001C0949A789428C001E0F894B0937D0080
:10106000EBE7F0E00093B3009598949862FF02C01C
:10107000C09A01C0AB9A789417C095FD0BC0F89444
:10108000B0937D00E5E7F0E0C09862FF01C0959A5B
:1010900078940AC0F894B0937D00E9E6F0E0959862
:1010A00062FF01C0C09A78946F7D089528E630E011
:1010B000F9012092B300C098AC989598AB98AD9880
:1010C00094986B7F0895A4EBB0E00FEF0D930D9310
:1010D0000D930D9303E00D9304E00D9309E00D9340
:1010E00003E00D9301E00D9301E00D93A0ECB0E05F
:1010F00001E00D930FEF0D930D930D930D930D9351
:1011000003E00D930FEF0D930FEF0D930D9305E299
:101110000D9300ED0D930AEF0D930AEF0D9304E08C
:101120000D930FEF0D9301E00D9300E00D930AE78F
:101130000D930FEF0D9300E00D9301E00D9300E090
:101140000D9303E00D9308952091BB008B7F233016
:1011500009F48460B091BC00B33019F09F7DB1FDFB
:1011600090629F7BB091BD00B1FD9064223011F080
:10117000886001C0877F08950A95E00FF21DB49141
:101180000895ECE1F0E00091B400F6DFB093D800F0
:10119000ECE1F0E00091B500EFDFB093D900EAE2B6
:1011A000F0E00091BA00E8DFB093DA00B091D0002F
:1011B0000FEF1CE0B23011F400EA1AE0B33011F482
:1011C00002E815E00093720010937300E8E3F0E08A
:1011D0000091D700D1DFB093A20008950895209127
:1011E000CA003091CB00B091BC00B33009F43E503E
:1011F00097FF02C020E03FEFB32FB21B6B2EB25817
:1012000010F4B2E86B2E00E00395609EB12DBD573F
:10121000D8F30093AE0008959068E1DF09DA20E08A
:1012200030E0B0E16B2E00DAB09197002B0F321D49
:101230006A94C9F7B4E036952795BA95E1F7822EFE
:101240009F77CDDF0895F894E3E0F0E0B9E0B7BF11
:10125000B491B078C1F3F894A895B1B5B861B1BDB7
:10126000B0E0B1BDB4E0BEBFBFE5BDBF1FDFB0E0C1
:10127000B8BBB1E1B7BBB0E0B5BBB8E3B4BBB0E05D
:10128000B2BBB0E3B1BB2224A0E0B0E02D92AA3102
:10129000E9F7A0E6B0E00FEF2D920A95E9F7B1E08B
:1012A000B093A40010DFEAD2B6B1B460B6B9009131
:1012B000CC000093AF00B1E0B0936A00F894BCD9C1
:1012C000C6D9B6D9C7D9B4D9C8D9B2D95ED3B4D9D9
:1012D000B3D9B0D9F8940AEF1AEFA0B396FDA09550
:1012E000A2FF1FC01A95C9F70A95B1F7E0E0FCE12B
:1012F000B591B43E39F4B591B03E21F4B591BF3FFC
:1013000009F40CC0E0E0F395F395B591B83F49F4CA
:10131000B591B43931F4B591BA3A19F4EE27F6958E
:10132000099412DF2EDF5ADF5ADF0091CC000093C0
:10133000AF00BCDEB2E0B3BFB2E0BEBDB2E0B5BD4F
:10134000B1E5B8BFB9BFB0B7B77FB0BFB8B1B0B73C
:10135000B860B0BF67D97894F5DAB3E096FDB2E033
:10136000B5BFB0E4BBBFBB27B064BABF8D7F64D943
:10137000626033E02CE0B0919600BB2321F42CE0B6
:101380003A9509F4A7CF54D980FFA4CF8E7FB091AE
:101390009700B23078F3B92FBF7100919900009394
:1013A0009800B0939900B01729F72A9521F76D7F1F
:1013B000B3E096FDB2E0B5BFBB27B064BABF8D7F86
:1013C000B091D600BB2321F48062B92FB0709B2F5F
:1013D0008F7B209267002ED985FF05C0B0916700F2
:1013E000BA3008F0806420D902E085FF01C000E037
:1013F000B0919700B017B8F3F89429D928D927D914
:1014000078941AD920928700B091BC00B33009F4C7
:1014100074C00AD9B091C000B13008F46EC0B09168
:101420006A00B13008F469C085FD18C0B09197001A
:10143000BF3F08F462C0F89413D97894FBD8B091F8
:101440009700B130C0F7F89402D9F0D800D9789459
:10145000F1D8B0919700BF3FB0F3C9C2B8E09B2E5E
:101460009068F894BCDE7894E5D8F8949F77B7DE5E
:1014700080909700B0919700BF37789408F445C0EA
:10148000D1D8F894EDD878949A9451F7C5DEB82D58
:10149000B550B093CB00D0D8F8941DD27BD27894BD
:1014A000BAE09B2E9068F8949ADE7894C3D8F894AA
:1014B0009F7795DE80909700B0919700BF37789422
:1014C00078F7B0D8F894C3D8B1D8C1D878949A94A2
:1014D00049F7A2DEB82DBB5FB093CA00ADD8F8942F
:1014E000FAD167D27894A6D8F89479DE7894B0913E
:1014F0009700BF3F08F498CF7AC200919700B0914F
:1015000087000B1710F00093870094D801E0B0918A
:10151000BC00B35009F405E0B0919700B01708F093
:1015200073CFF8949DD89CD89BD8789485D8209276
:101530006A0020926B0020926C00B0916B00B39512
:10154000B0936B00BF3F69F5B0916C00B395B09359
:101550006C00B091CE0009E1BA9559F002E3BA955A
:1015600041F00DE7BA9529F00AEFBA9511F02092F3
:101570006C00B0916C00B017A0F0B0916C00BA95FF
:10158000B0936C00B4EBB0936B00B091CD00B0930E
:10159000AF00F89465D87894B091CC00B093AF00C8
:1015A00049D844D8B0916800BB2319F485FF01C025
:1015B00091CE01E085FD01C006E0B0919700B01723
:1015C00008F4BBCFB091BC00B35009F033D8B09150
:1015D0006800BB2309F47ECEF89468DD2092610098
:1015E0002092620020926300522C2092640020928C
:1015F000A3007894B091B900BB0FB093A0002092E3
:101600007F00209280002092810020928200209210
:1016100083002092AC0060E070E020927100B8E09E
:10162000B093AC007860FED7B2E073FDB1E0B7B91B
:10163000B6B1B068B064B6B9B6B1B6FDFDCF04B10D
:1016400015B1B6B1BF77B6B9112309F00FEF00930A
:10165000AD007AD9B8E0B093AC0078608090BB0060
:10166000B2E0B093BB0070DD8092BB00F894BFEF96
:10167000B0939C00B2D9B0916100B0939C00B0933C
:101680009D00B0939E007894B1E0B0936100B09358
:1016900063005B2EB0936400B093A600B0919B00F2
:1016A000B093A500B091BC00B33019F49F7D87FDC5
:1016B00090627160726020926D00A5DCB6DCA6D9E4
:1016C000ABD9A4D9A9D9A2D906C0F8943DDD7894A4
:1016D0002092AC00777F0EDB3AD8C0DBF0DB9CD9E0
:1016E00002DB66FD35D876FFEDD876FD1BD9B6DB7B
:1016F000F8DB92D9FFDA66FD4DD8B0DB32DC8CD94D
:10170000F2DA66FD81D8AADB3EDC86D9F3DA66FD23
:10171000ABD8A4DB78DC80D9E6DAB2E073FDB1E0C7
:10172000B7B9B6B1B068B064B6B998DB7EDC74D92D
:101730000BD971FF23C067FD21C0B0919F00B0930A
:101740009C00B0939D00B0919B00B093A500B1E0C8
:10175000B093A60018E12CE0B0916D00B11740F0F5
:101760007D7F746020936F00BFEFB0939C0006C034
:10177000B0919700B13008F0AECF5AC072FF10C0E0
:1017800067FD0EC0B0916F00BA9511F47B7F9DCFBD
:10179000B0936F00B0919700B13008F09CCF48C073
:1017A00020927000B0919A0002E8B01708F040C093
:1017B00085FF04C0B0916800BB23D1F1B091BC009B
:1017C000B33081F495FD03C087FD04C00BC087FFD3
:1017D00001C008C067FD06C06068B0919F00B0936B
:1017E0009C008ECF00EF67FF05C0B0919F00B093C3
:1017F0009C0000E2B0917B00B01708F46CCF67FF4B
:1018000017C06F779F7D87FD90627460B2E1B093DF
:101810006F00B0919F00B0939C005DCFB0917000BD
:10182000B395B0937000B0919700BB2309F002C04C
:1018300020927000F8943ADC8090BB00B2E0B09344
:10184000BB0082DC8092BB0020926100209262008B
:1018500020926300522C209264002092A0007E7F90
:101860007894E0D623DCB6B1B460B6B985FF05C084
:10187000B0917000B53008F02DCD5BCEEDE0F0E01A
:1018800023D00A3509F01BC0EEE0F0E01DD0053A88
:1018900009F015C03AE0A4EBB0E0E3E0F0E014D0CA
:1018A0000D9331963A95D9F738E1A0ECB0E0EFE02E
:1018B000F0E00AD00D9331963A95D9F702C003DCD7
:1018C0000AD0E7E2F0E00895E199FECFEEBBFFBB5E
:1018D000E09A0DB308951ED03AE0A4EBB0E0E3E047
:1018E000F0E00D910FD031963A95D9F738E1A0ECA0
:1018F000B0E0EFE0F0E00D9105D031963A95D9F7E0
:1019000012D00895E199FECF0DBBEEBBFFBBE29A6A
:10191000E19A0895EDE0F0E00FEFF4DFEEE0F0E0A3
:101920000FEFF0DF0895EDE0F0E00AE5EBDFEEE029
:10193000F0E005EAE7DF08953091B0000091B100D2
:10194000313011F40093B800323011F40093B90033
:10195000333011F40093BA00343011F40093C60010
:10196000353011F40093BB00363011F40093D700EA
:10197000373011F40093D000383011F40093BC00DC
:10198000393011F40093BD00089525E055D62A950D
:10199000E9F708955CD65ED660D662D647D657D6AC
:1019A00059D65BD65DD642D652D654D656D658D6E0
:1019B000089556D652D64ED64AD638D651D64DD69A
:1019C00049D645D633D64CD648D644D640D60895C7
:1019D0008090B0009090B1003AD639D638D626D64D
:1019E0008A94D1F73DD622D69A94E1F70895F894D7
:1019F000D1DF7894CADFC9DFB1E0B093B000B1E0C5
:101A0000B093B1002092B200F894E2DF7894B5E090
:101A10006B2E7090970010D6B09197007B16C9F787
:101A2000B13018F0BF3F40F107C086DFF89453DFB4
:101A3000B1DFB8E0B1BDA9DF6A9459F7B091B20047
:101A4000B395B093B200B33008F4DECF9EDFB0910F
:101A5000B100B395B093B100F894B091B000BA95CD
:101A6000EEE3F0E0EB0FF21D049178940395B09152
:101A7000B100B01708F4C6CF88DF87DFB091B0009F
:101A8000B395B093B000B091B000BA3008F4B7CFBE
:0E1A90001ADBF89420DFB8E0B1BD77DFD4CBCD
:00000001FF
